:100000000C9471080C9491080C9491080C9491082C
:100010000C9491080C9491080C9491080C949108FC
:100020000C9491080C9491080C9491080C949108EC
:100030000C9491080C9491080C9491080C949108DC
:100040000C9491080C9480130C9491080C949108D2
:100050000C9491080C9491080C9491080C949108BC
:100060000C9491080C94F22B0C94BE2B0C949108D8
:100070000C9491080C94A2080C9491080C9491088B
:100080000C9491080C9491080C9491080C9491088C
:100090000C9491080C9491080C9491080C9491087C
:1000A0000C9491080C9491080C9491080C9491086C
:1000B0000C9491080C9491080C9491080C9491085C
:1000C0000C9491080C9491080C9491080A73772071
:1000D000310A000A737720300A00414D433A206EFE
:1000E0006F77204D300A00414D433A206E6F7720E4
:1000F0004D310A00414D433A2068616E646C6520C1
:10010000636C6F7365640A00414D433A204D3120A2
:1001100068616E646C652073746174757320636FBD
:100120007272656374696F6E0A00414D433A206EC6
:100130006F77204D320A00414D433A2068616E646A
:100140006C65206F70656E65640A00414D433A200E
:100150006E6F77204D330A00414D433A2068616E3F
:10016000646C65206F70656E65640A00414D433AAA
:10017000206E6F77204D340A00414D433A2068616C
:100180006E646C65206F70656E65640A00414D4356
:100190003A204D342068616E646C6520737461741C
:1001A000757320636F7272656374696F6E0A0041C4
:1001B0004D433A206E6F77204D350A00414D433A4A
:1001C0002068616E646C6520636C6F7365640A00FF
:1001D000414D433A206E6F77204D360A000A414D5B
:1001E00043206873776170206F75743A20000A535A
:1001F0004953383330300A004275696C742077698E
:100200007468204156522D4743433A2000342E361D
:100210002E320020616E64204156522D4C494243DB
:100220003A2000312E382E30002072656C656173E3
:10023000653A20003230313131323238000A6F6E87
:1002400020004F6374203136203230313400202FAB
:10025000200030373A30323A3336000A0A00414D36
:1002600043207374617475733A204D000A00525430
:100270004D207374617475733A204D000A0A002092
:10028000436F6D6D616E646C6973743A0A205354E8
:100290004154202D204669726D7761726520526548
:1002A000766973696F6E2C205374617475732C209A
:1002B0006574632E2E2E0A2048454C50202D207444
:1002C00068697320706167650A002072746D207A16
:1002D0006F6E65333A200020616D63207A6F6E6522
:1002E000333A20002072746D206D617463683A2087
:1002F000002072746D20636C6F7365640A00207255
:10030000746D206F70656E65640A002072746D20D4
:100310006F70656E65640A002072746D206F706581
:100320006E65640A002072746D206F70656E65647E
:100330003A2000505752202B3132563A2000206D7F
:10034000560A4420202B332E33563A202000206DAD
:10035000560A4420202B312E30563A202000206DA2
:10036000560A4420202B312E38563A2020002045B2
:1003700072617375726520454550524F4D202E2E87
:100380002E2000205772697465204144353333387C
:100390003A200020526561642041443533333800EF
:1003A00069326320627573206572726F720A00751C
:1003B0006E6B6E6F776E2069326320737461746543
:1003C0002000657272207374613A20006572722099
:1003D000736C613A2000657272206474613A200087
:1003E0000A0A5349533833303020646562756720F8
:1003F00070726F6D70740A000A0A626F6F747661B2
:100400006C7565203D20000A000A00574454435390
:10041000523A20000A004D4D432046573A20000A28
:100420004275696C742077697468204156522D4773
:1004300043433A2000342E362E320020616E642071
:100440004156522D4C4942433A2000312E382E302D
:10045000002072656C656173653A2000323031317D
:1004600031323238000A6F6E20004F63742031360B
:10047000203230313400202F200030373A30323AE9
:100480003339000A004D435553523A20000A007296
:1004900065737461727420616674657220636F6C39
:1004A000642072657365740A004D4F44535441547F
:1004B000455F504F5745524544202D3E204D4F44F7
:1004C00053544154455F574149545F524553455435
:1004D00020000D0A004D4F4453544154455F57418D
:1004E00049545F5245534554202D3E204D4F4453AF
:1004F000544154455F574149545F465047415F441A
:100500004F4E4520000D0A004D4F44535441544571
:100510005F574149545F465047415F444F4E452025
:100520002D3E204D4F4453544154455F4650474162
:100530005F52445920000D0A004D4F44535441541A
:10054000455F465047415F52445920000D0A0070F4
:100550008A728E9290748C76989C9AA0A4889E86BB
:100560008478947A9682807C7EA2070051013100C3
:100570000006C10003540201FF7F00703F00000429
:100580000000620200040CC0077FEFABFF00F7F22F
:10059000E9A2A7AB0202000000C6442B312E385658
:1005A00000000000000000000000060051013100C2
:1005B0000005C10003540201FF7F00703F000004EA
:1005C0000000620200040CC0077FEFABFF008E84C6
:1005D0007A42484D0202000000C6442B312E3056AC
:1005E0000000000000000000000002005101300087
:1005F0000001C10003550101FF7F00703F00800131
:100600000000010600040C00001946007DC9555089
:100610004600050A0505000000C574465047410024
:100620000000000000000000000000005111150053
:1006300001002B000000C00000CA5349533833307A
:100640003052544D00005112120000002B000000E7
:10065000C10000C753495338333030020051012FD5
:10066000000008C00003540101FF7F00703F0080BC
:10067000010000010600040C00001946007DC95568
:10068000463C00050A0505000000C47452544D00A4
:1006900000000000000000000000000100510135D2
:1006A000000007C0000340F26F07000000070000D1
:1006B000000000000000000000000000000000003A
:1006C00000000000000000000000CA486F7453776B
:1006D000617052544D0000000000000500510131CE
:1006E000000004C10003540201FF7F00703F0000BE
:1006F000040000A10200040CC0077FEFABFF00F76D
:10070000F2E9A2A7AB0202000000C6442B332E334D
:1007100056000000000000000000000400510132FB
:10072000000003C10003540201FF7F00703F00007E
:10073000040000360200040CD0077FEFABFF00F787
:10074000F2E9A2A7AB0202000000C75057522B31BA
:10075000325600000000000000000003005101318B
:10076000000002C10003540101FF7FFF7F3F0080B2
:10077000010000010600040C0000193C3278E75526
:10078000463C00050A0505000000C674506F7765F9
:100790007200000000000000000000010051013262
:1007A000000000C1000340F26F07000000070000D6
:1007B0000000000000000000000000000000000039
:1007C00000000000000000000000C7486F7453776D
:1007D000617000000000000000000070726F633A5A
:1007E000204E4554464E5F4150503A20434D445FA1
:1007F0004745545F4445564943455F49440A0070A4
:10080000726F633A204E4554464E5F53454E535FD8
:100810004556454E543A20434D445F5345545F4539
:1008200056454E545F52454345495645520A00705D
:10083000726F633A204E4554464E5F53454E535FA8
:100840004556454E543A20434D445F4745545F4515
:1008500056454E545F52454345495645520A00702D
:10086000726F633A204E4554464E5F53454E535F78
:100870004556454E543A20434D445F504C415446F2
:100880004F524D5F4556454E540A0070726F633AA1
:10089000204E4554464E5F53454E535F4556454E98
:1008A000543A20434D445F4745545F4445564943BD
:1008B000455F5344525F494E464F0A0070726F6362
:1008C0003A204E4554464E5F53454E535F4556457C
:1008D0004E543A20434D445F4745545F4445564982
:1008E00043455F5344520A0070726F633A204E458D
:1008F00054464E5F53454E535F4556454E543A203D
:10090000434D445F5245535F4445564943455F5309
:1009100044525F5245500A0070726F633A204E4550
:1009200054464E5F53454E535F4556454E543A200C
:10093000434D445F4745545F53454E534F525F52BA
:10094000454144494E470A0070726F633A204E4554
:1009500054464E5F53454E535F4556454E543A20DC
:10096000434D445F4745545F53454E534F525F5488
:1009700048524553484F4C44530A0070726F633AD3
:10098000204E4554464E5F53454E535F4556454EA7
:10099000543A20756E6B6E6F776E3A200070726FEE
:1009A000633A204E4554464E5F53544F524147459B
:1009B0003A20434D445F4745545F4652555F494E88
:1009C000565F415245415F494E464F0A0070726F73
:1009D000633A204E4554464E5F53544F524147456B
:1009E0003A20434D445F524541445F4652555F446F
:1009F0004154413A2000414D430A0052544D0A00EF
:100A000070726F633A204E4554464E5F53544F52B6
:100A10004147453A20434D445F57524954455F464C
:100A200052555F444154413A2000414D430A00521F
:100A3000544D200070726F633A204E4554464E5F0D
:100A40005049434D473A20434D445F4745545F501A
:100A500049434D475F50524F50530A0070726F63C5
:100A60003A204E4554464E5F5049434D473A204345
:100A70004D445F4652555F434F4E54524F4C3A20BF
:100A800000414D430A0052544D0A0070726F633AA0
:100A9000204E4554464E5F5049434D473A20434D02
:100AA000445F4745545F4652555F4C45445F505242
:100AB0004F50530A0070726F633A204E4554464EB1
:100AC0005F5049434D473A20434D445F4745545F8B
:100AD0004C45445F434F4C4F525F43415041420AA3
:100AE0000070726F633A204E4554464E5F50494342
:100AF0004D473A20434D445F5345545F4652555F3E
:100B00004C45445F53544154450A0070726F633A38
:100B1000204E4554464E5F5049434D473A20434D81
:100B2000445F4745545F4652555F4C45445F5354BC
:100B30004154450A0070726F633A204E4554464E48
:100B40005F5049434D473A20434D445F4745545F0A
:100B50004652555F4C45445F53544154452065729D
:100B6000723A000A0070726F633A204E4554464E46
:100B70005F5049434D473A20434D445F4745545FDA
:100B80004445565F4C4F4341545F5245435F49448F
:100B90000A0070726F633A204E4554464E5F5049CA
:100BA000434D473A20434D445F4652555F434F4EB5
:100BB00054524F4C5F43415041420A0070726F6380
:100BC0003A204E4554464E5F5049434D473A2043E4
:100BD0004D445F5345545F414D435F504F52545F06
:100BE00053544154450A0070726F633A204E455485
:100BF000464E5F5049434D473A20434D445F474579
:100C0000545F414D435F504F52545F5354415445DC
:100C10000A0070726F633A204E4554464E5F504949
:100C2000434D473A20434D445F4745545F434C4F43
:100C3000434B5F53544154450A0070726F633A202E
:100C40004E4554464E5F5049434D473A20434D442C
:100C50005F5345545F4652555F4143544956415492
:100C6000494F4E0A0070726F633A204E4554464E0B
:100C70005F5049434D473A20434D445F5345545FCD
:100C8000504F5745525F4C4556454C0A0070726FA5
:100C9000633A204E4554464E5F5049434D473A20F3
:100CA000756E6B6E6F776E0A0070726F633A204ECE
:100CB0004554464E5F56454E444F523A20434D44AC
:100CC0005F524541445F52544D5F45450A00707282
:100CD0006F633A204E4554464E5F56454E444F5240
:100CE0003A20434D445F57524954455F52544D5F3B
:100CF00045450A0070726F633A204E4554464E5F78
:100D000056454E444F523A20434D445F4D4F44495F
:100D100046595F52544D5F45455F57500A00707207
:100D20006F633A204E4554464E5F56454E444F52EF
:100D30003A20434D445F5345545F464C4153485F0E
:100D4000424F4F545F5245560A0070726F633A200B
:100D50004E4554464E5F56454E444F523A20434D01
:100D6000445F52455345545F465047410A007072F4
:100D70006F633A204E4554464E5F56454E444F529F
:100D80003A20434D445F4745545F4649524D575FB3
:100D900056455253494F4E0A0070726F633A204EC7
:100DA0004554464E5F56454E444F523A20434D44BB
:100DB0005F4745545F754457435F4441435F564125
:100DC0004C55450A0070726F633A204E4554464EAA
:100DD0005F56454E444F523A20434D445F5345546D
:100DE0005F754457435F4441435F56414C55450A44
:100DF0000070726F633A204E4554464E5F56454E22
:100E0000444F523A20434D445F524541445F52544F
:100E10004D5F54454D505F56414C55450A00707228
:100E20006F633A204E4554464E5F56454E444F52EE
:100E30003A20434D445F5345545F52544D5F5445EF
:100E40004D505F504F494E0A0070726F633A204E0A
:100E50004554464E5F56454E444F523A20464F4FFA
:100E6000200A0052544D3A206E6F77204D300A0010
:100E700052544D204D61736B3A200052544D3A202C
:100E80004552524F523A20493243206275732053E3
:100E9000444120737475636B206C6F770A00525461
:100EA0004D3A20636F6D7061746962696C69747921
:100EB00020636865636B3A20006D730A0052544DDD
:100EC0003A206E6F77204D310A00636F6D702E20CF
:100ED000636865636B3A20737563636573730A00B7
:100EE000636F6D702E20636865636B3A206E6F20B0
:100EF0006D61746368657320666F756E640A005275
:100F0000544D204D61736B3A20000A0052544D3A03
:100F10002068616E646C6520636C6F7365642C205F
:100F2000656467650A0052544D3A2068616E646CCE
:100F30006520636C6F7365642C204D30206C657682
:100F4000656C0A0052544D3A206D6F64756C6520D3
:100F500072656D6F7665640A0052544D3A206E6F6B
:100F600077204D320A0052544D204D61736B3A2068
:100F70000052544D3A2068616E646C65206F706554
:100F80006E65640A0052544D3A206D6F64756C654D
:100F90002072656D6F7665640A0052544D3A206E7A
:100FA0006F77204D330A0052544D3A206E6F7720F0
:100FB0004D340A0052544D204D61736B3A2000525B
:100FC000544D3A205365747570204457435F444133
:100FD0004320746F203256350A0052544D3A20682F
:100FE000616E646C65206F70656E65640A005254B2
:100FF0004D3A206D6F64756C652072656D6F766516
:10100000640A0052544D3A20536574646F776E2021
:101010004457435F4441430A0052544D3A206E6F97
:1010200077204D350A0052544D204D61736B3A20A4
:101030000052544D3A20536574646F776E204457C4
:10104000435F4441430A0052544D3A206D6F64752A
:101050006C652072656D6F7665640A0052544D3A76
:10106000206E6F77204D360A0052544D204D61732B
:101070006B3A200052544D3A206D6F64756C6520B8
:1010800072656D6F7665640A000A616D6320776929
:1010900074686F7574207A33207265636F7264733D
:1010A0000A000A72746D20776974686F7574207A0B
:1010B00033207265636F7264730A000A666F722070
:1010C000616D633A2000666F722072746D3A200081
:1010D0000A52544D206873776170206F75743A20FE
:1010E000000011241FBECFEFD1E2DEBFCDBF13E061
:1010F000A0E0B2E0E8E2F0E600E00BBF02C007903B
:101100000D92A03DB107D9F71BBE1AE0A0EDB3E0E8
:1011100001C01D92AE35B107E1F70E94DA2C0C94A4
:1011200012300C94000010920E0410927C0087EC98
:1011300080937A0080917A0084FFFCCF8FEC8093BB
:101140007A0008951F920F920FB60F920BB60F926E
:1011500011242F934F935F936F937F938F939F935C
:10116000AF93BF93EF93FF938091780090917900B4
:10117000A0E0B0E04091D0035091D1036091D20340
:101180007091D303840F951FA61FB71F8093D003C0
:101190009093D103A093D203B093D3032091D403AF
:1011A0002F5F2093D4032223E9F420910E04E22F31
:1011B000F0E0EE0FFF1FEA5FFB4F892F9A2FAB2F56
:1011C000BB27918380831092D0031092D103109299
:1011D000D2031092D303822F8F5F837080930E040B
:1011E00080937C008FEC80937A00FF91EF91BF9108
:1011F000AF919F918F917F916F915F914F912F91BF
:101200000F900BBE0F900FBE0F901F901895E82FF8
:10121000F0E0E370F070EE0FFF1FEA5FFB4F80819C
:10122000918108951F93CF93DF93CDB7DEB7C35459
:10123000D0400FB6F894DEBF0FBECDBF182F8DED96
:1012400091E00E942C2C812F0E94A52C80E092E03E
:101250000E941A2C809137098C8380E18D838091C4
:10126000EC088F838091360988878C5F80933609DC
:1012700082E0898784E08A8782EF8B871C868FE6ED
:101280008D871E878BE08B83CE0101960E943814D8
:1012900081E08A83CE0101960E94FA101093020227
:1012A000CD5BDF4F0FB6F894DEBF0FBECDBFDF9131
:1012B000CF911F910895CF9380E80E942B2BC82FC8
:1012C00080910402809303028091DB0380930402E7
:1012D0008091DC03C81749F0CC2319F08CEC90E026
:1012E00002C083ED90E00E942C2C80E80E942B2B02
:1012F0009091DA03882319F09D7F916002C092607B
:101300009E7F9093DA0380910402833009F482C0B7
:10131000843040F490910302813071F1823008F002
:1013200058C00AC0853009F4D3C0853008F498C08D
:10133000863009F00DC1F0C0992309F406C18AED89
:1013400090E00E942C2C80E060E041E050E00E94A0
:10135000381181E060E041E050E00E94381182E005
:1013600060E043E050E00E94381182E060E040E03D
:1013700050E00E943811E9C0913051F080E060E007
:1013800041E050E00E94381187EE90E00E942C2C42
:101390008091DC03C81771F0CC2361F0C093DC03AB
:1013A00084EF90E00E942C2C80E00E94120982E0E1
:1013B0008093DB038091DC03C81709F445C0CC237C
:1013C00009F042C01092DC0388E091E00E942C2CCE
:1013D0003BC0923021F08AE291E00E942C2C809157
:1013E000DC03C81771F0CC2361F41092DC0387E3AF
:1013F00091E00E942C2C81E00E94120981E08093F0
:10140000DB038091D903882309F4A2C01092D90389
:1014100083E09CC080910302833021F08BE491E053
:101420000E942C2C8091DC03C81771F0CC2361F44E
:101430001092DC0388E591E00E942C2C81E00E9450
:10144000120981E08093DB038091D803882309F49B
:101450007FC01092D80381E08093EB0884E076C0CF
:1014600080910302843021F08CE691E00E942C2CC4
:101470008091DC03C81781F0CC2371F41092DC0357
:1014800089E791E00E942C2C81E00E94120985E0FE
:101490008093DB031092E3088091DC03C81741F0CE
:1014A000CC2331F0C093DC038DE891E00E942C2C1A
:1014B0008091D603882309F44BC01092D60387E0AD
:1014C0008093EB0886E08093DB031092E30840C032
:1014D00080910302853021F08FEA91E00E942C2C4C
:1014E0008091DC03C81771F0CC2361F0C093DC035A
:1014F0008CEB91E00E942C2C80E00E94120984E089
:101500008093DB038091D703882379F01092D7036F
:1015100086E08093DB0309C080910302863029F0C6
:101520000D9A80ED91E00E942C2C8091D6038823A7
:1015300029F01092D60387E08093EB088091EB08A6
:10154000882331F482E00E94120981E08093DB035A
:101550008091D503882329F18091DA0380FF03C0AD
:1015600080E00E9412098091DA0381FF03C081E0CC
:101570000E9412098091DA0382FF03C082E00E9478
:1015800012098091DA0383FF03C083E00E941209ED
:101590008091DA0384FF03C084E00E941209109254
:1015A000D503CF9108958091040208958091DA03C4
:1015B000089581E08093D903089581E08093D80352
:1015C0001092D7031092D603089581E08093D70339
:1015D0001092D8031092D603089581E08093D60329
:1015E0001092D7031092D803089581E08093D50319
:1015F00008956F927F928F929F92AF92BF92CF92F7
:10160000DF92EF92FF920F931F93CF93DF93CDB7AB
:10161000DEB7C850D1400FB6F894DEBF0FBECDBFC5
:101620004C01E62E3A01FC011082CE01019660E0E9
:1016300070E048E050E00E94E22FFE01319697E012
:1016400080E02191820F9150E1F78195988589176B
:1016500009F059C00E8110E093E0000F111F9A9518
:10166000E1F70115110509F450C089E0A82EB12C4D
:10167000AC0EBD1EB80160507040CE01019645E031
:1016800050E00E94E22F8A819981890FFB808F0DA3
:101690009C81890F81959D818917C9F5CF2CDD2407
:1016A0000B5F1F4FB80160507040C501A6010E943A
:1016B000E22F20E030E006C08A0D9B1DFC018081F6
:1016C000280F3F5F832F90E08C159D05A8F321958F
:1016D0008C812817F1F48C85803379F4F4018081B2
:1016E0008F5F80838E1549F46114710431F0C3015A
:1016F000B5014F2D50E00E94D92F8A8187FD0BC084
:101700000C0D1D1DB7CF82E007C083E005C084E04B
:1017100003C085E001C080E0C85FDE4F0FB6F894DB
:10172000DEBF0FBECDBFDF91CF911F910F91FF9014
:10173000EF90DF90CF90BF90AF909F908F907F9071
:101740006F900895EF92FF920F931F93CF93DF93C3
:10175000CDB7DEB728970FB6F894DEBF0FBECDBF6A
:101760007C01CE01019660E070E048E050E00E940C
:10177000E22FFE01319697E080E02191820F915097
:10178000E1F781959885891749F50E8110E023E0EE
:10179000000F111F2A95E1F70115110509F1B80194
:1017A00060507040CE01019645E050E00E94E22F6B
:1017B0002A819981920F8B81980F3C81930F91958B
:1017C0003D81931779F490E00596080F191F27FFC4
:1017D000E6CFF7011183008380E005C082E003C0FB
:1017E00083E001C084E028960FB6F894DEBF0FBEF8
:1017F000CDBFDF91CF911F910F91FF90EF90089592
:1018000088E193E00E942C2C80E008958FE792E01D
:101810000E942C2C80E00895CF93DF9300D0CDB7A9
:10182000DEB783E993E00E942C2C8CE061E0AE01EE
:101830004F5F5F4F0E940D29882329F085E092E0D9
:101840000E941A2C0AC08DE092E00E941A2C898115
:101850000E94A52C8A810E94A52C82E192E00E9420
:101860001A2C80E00F900F90DF91CF910895CF93C5
:10187000DF9300D000D0CDB7DEB719821A821B8269
:101880001C828CE289838CE18A83A5E4B4E0FE01AA
:10189000319680E090E03D91232F20532A3008F0CC
:1018A00027502193019684309105A9F7898182956B
:1018B000807F9A819F70892B89838B818295807F1D
:1018C0009C819F70892B8A8383E893E00E942C2C53
:1018D00089810E94A52C8A810E94A52C8CE061E060
:1018E000AE014F5F5F4F0E94F525882319F084E118
:1018F00092E002C080E292E00E941A2C80E00F90F9
:101900000F900F900F90DF91CF910895CF93DF93B9
:101910008EE693E00E942C2CC0E0D0E080E5BE0172
:1019200040E00E94FB24219682E0C030D807B1F746
:101930008BE292E00E941A2C80E0DF91CF91089513
:10194000EF92FF920F931F93CF93DF9300D000D0BD
:1019500000D0CDB7DEB782E392E00E941A2C81E579
:101960006AEF70E046E050E09E012F5F3F4F0E941B
:101970005825882329F084E492E00E941A2C10C094
:101980007E010894E11CF11C00E010E0F701819158
:101990007F010E94A52C0F5F1F4F06301105B1F784
:1019A00082E192E00E941A2C80E026960FB6F8940D
:1019B000DEBF0FBECDBFDF91CF911F910F91FF9082
:1019C000EF900895CF93DF9380E00E940709EC0128
:1019D00083E393E00E942C2CBE0180E090E024E69B
:1019E0003DE84DE050E00E94712F0E945C2C81E0A8
:1019F0000E940709EC018EE393E00E942C2CBE01AB
:101A000080E090E022E836E044E050E00E94712F50
:101A10000E945C2C82E00E940709EC018EE493E0B6
:101A20000E942C2CBE0180E090E026E536E040E0EC
:101A300050E00E94712F0E945C2C83E00E940709F5
:101A4000EC018EE593E00E942C2CBE0180E090E03A
:101A500020E13AE340E050E00E94712F0E945C2CAC
:101A60008EE492E00E941A2C80E0DF91CF910895DD
:101A7000EF92FF920F931F93CF93DF9300D0CDB7D8
:101A8000DEB785E293E00E942C2CCE0101960E94E5
:101A9000FD2290E00E945C2C03E512E0C8010E9448
:101AA0001A2C89819A810E945C2C22E1E22E22E08C
:101AB000F22EC7010E941A2CCE0101960E94A20BA1
:101AC00090E00E945C2CC8010E941A2C89819A81A6
:101AD0000E945C2CC7010E941A2C80E00F900F908E
:101AE000DF91CF911F910F91FF90EF9008958BE0C0
:101AF00093E00E942C2C86E00E94942080E00895C0
:101B00008EEF92E00E942C2C81E00E94942080E0D5
:101B1000089581EF92E00E942C2C80E00E94942096
:101B200080E0089584EE92E00E942C2C0E941624FE
:101B300090E00E945C2C82E192E00E941A2C88E0E6
:101B40000E94942080E00895CF93DF930F92CDB749
:101B5000DEB787ED92E00E942C2CCE01019660E06A
:101B600040E050E00E94F90A90E00E945C2C83E57E
:101B700092E00E941A2C898190E00E945C2C82E104
:101B800092E00E941A2C87E00E94942080E00F903F
:101B9000DF91CF910895CF93DF930F92CDB7DEB74A
:101BA0008AEC92E00E942C2CCE01019660E040E08D
:101BB00050E00E946B2390E00E945C2C83E592E051
:101BC0000E941A2C898190E00E945C2C82E192E0B4
:101BD0000E941A2C85E00E94942080E00F90DF91F3
:101BE000CF9108958EEE91E00E942C2C88EF91E029
:101BF0000E942C2C8DE092E00E942C2C83E192E03C
:101C00000E942C2C83E292E00E942C2C89E292E02C
:101C10000E942C2C84E392E00E942C2C8DE392E015
:101C20000E942C2C82E492E00E942C2C8EE492E004
:101C30000E942C2C82E592E00E942C2C8BE592E0F5
:101C40000E942C2C8EE592E00E942C2C0E94D30A3C
:101C500090E00E945C2C8CE692E00E942C2C8EE698
:101C600092E00E942C2C0E947C2090E00E945C2C30
:101C70008CE792E00E942C2C80E0089585E592E0AC
:101C80000E941A2C10923F040895CF93DF93AC0169
:101C9000A0E08A2F90E0880F991F880F991FFC0100
:101CA000E154FD4F60817181B0E02B2F30E0FB01EA
:101CB000E20FF31FE081EE2359F0240F351FE901F5
:101CC00028812E272F7511F4BF5FEFCFAF5FE1CFD3
:101CD000BB2349F081549D4FDC011296ED91FC919C
:101CE0001397099501C081E0DF91CF910895CF93BB
:101CF000DF930F92CDB7DEB7CE0101960E94A02BE5
:101D0000882309F04CC08981883019F08D3081F525
:101D100010C080913F04882309F441C08150809312
:101D20003F0488E00E94812B80E20E94812B88E0A2
:101D300034C08AE00E94812B8DE00E94812BE091CB
:101D40003F04EE2371F0F0E0E05CFB4F108280E492
:101D500094E00E94450E882321F08EE592E00E94D7
:101D60001A2C10923F048FE692E00E941A2C17C0A2
:101D70008B31A9F090913F04903270F40E94812B36
:101D800080913F04E82FF0E0E05CFB4F9981908365
:101D90008F5F80933F0403C087E00E94812B0F90E8
:101DA000DF91CF9108950F931F93CF93DF93C6E3F5
:101DB000D0E0CE010E94F22F90E08F70907024E668
:101DC00030E0829F8001839F100D929F100D11249F
:101DD000CE0101960E94F22F90E08F7090709C01CE
:101DE000220F331F53E0880F991F5A95E1F7280FF0
:101DF000391F020F131FCE0102960E94F22F8F701F
:101E00009801280F311DC901DF91CF911F910F91CA
:101E10000895CF92DF92EF92FF920F931F9386E384
:101E200090E00E94F22F90E08F70907024E630E0F6
:101E3000829F6001839FD00C929FD00C1124EE24CE
:101E4000D7FCE094FE2C87E390E00E94F22F90E014
:101E50008F7090709C01220F331F63E0880F991FD1
:101E60006A95E1F7280F391FC901AA2797FDA095A8
:101E7000BA2FC80ED91EEA1EFB1E88E390E00E940E
:101E8000F22F8F70A7019601280F311D411D511DA2
:101E9000DA01C9015A98EFE9FFE03197F1F700C084
:101EA00000005A9AE0E2F0E000E010E020E030E8C4
:101EB0005B98B901A801482359236A237B23411564
:101EC00051056105710509F05B9AF8945A985A9A80
:101ED00078943695279517950795319749F71F916F
:101EE0000F91FF90EF90DF90CF90089590E2909344
:101EF000B8008E7F8093BA001092BD0084E4809376
:101F0000BC0010926A04109269040895CF938091E6
:101F1000BC0087FF67C0C091B900C87FC03661F0C0
:101F2000C13620F4CC2309F448C051C0C038D1F0E8
:101F3000C03A09F04CC02BC01092DF03E091F108C9
:101F4000F091F20880818068808380818E7F808319
:101F50008091BB00838381E08093DF0394EC9093B6
:101F6000BC0012C0E091F108F091F2088091DF030B
:101F70009091BB00E80FF11D93838F5F8093DF0387
:101F800084EC8093BC0081E08093DE032BC0E09161
:101F9000F108F091F2088091DF03828380818160F3
:101FA000808380818F77808384EC8093BC00109243
:101FB000DE038AE080931A0315C080EA93E00E9452
:101FC0002C2C8091BC0080698093BC000BC08FEAF0
:101FD00093E00E942C2C8C2F0E94A52C8FEF92E076
:101FE0000E941A2C8091DE03CF910895CF92DF9248
:101FF000FF920F931F93CF93DF930F92CDB7DEB76E
:102000008091DD03882341F490916A0480916904F2
:10201000981709F053C0E5C08F3F39F484E60E9459
:102020004C2B8EEF8093DD03DCC08E3F09F046C061
:1020300080919B08882311F14091690450E023E4CA
:1020400030E0429FC001439F900D529F900D11249C
:1020500085599B4F0E94442090916804891771F420
:10206000809169048F5F80936904803111F410922C
:1020700069041092DD0310929B08B3C00E945C2B90
:10208000882309F4AEC08091E00381508093E0037F
:10209000882321F084E60E944C2B10C080916904B3
:1020A0008F5F80936904803111F41092690481E09C
:1020B00093E00E941A2C1092DD0393C084EA80936F
:1020C000BC008091BC0087FFFCCF1091B900187F45
:1020D000183059F082EC93E00E942C2C812F0E9442
:1020E000A52C8FEF92E00E941A2C2091690430E019
:1020F00083E490E0289FF001299FF00D389FF00DB8
:102100001124E559FB4F83818093BB0084E88093C1
:10211000BC008091BC0087FFFCCF1091B900187FF4
:10212000183159F08CEC93E00E942C2C812F0E94E6
:10213000A52C8FEF92E00E941A2C11E083E4C82EA8
:10214000D12C94E8F92E04E923C0181719F4009350
:10215000BC001DC0E10FF11D83818093BB00F09294
:10216000BC008091BC0087FFFCCF2091B900287F84
:10217000283269F086ED93E029830E942C2C298176
:10218000822F0E94A52C8FEF92E00E941A2C1F5FD5
:1021900020916904822F90E08C9DF0018D9DF00DBF
:1021A0009C9DF00D1124E559FB4F8281811768F643
:1021B0008181813059F48091DD038E3F79F08FEF7A
:1021C0008093DD0383E08093E00308C0822F8F5F5C
:1021D00080936904803111F41092690484EC809337
:1021E000BC000F90DF91CF911F910F91FF90DF9076
:1021F000CF90089560916A04462F50E023E430E0C8
:10220000429FF001439FF00D529FF00D1124E559BC
:10221000FB4FDC0183E40D9001928150E1F76F5F89
:1022200060936A04603111F410926A0480E00895AA
:1022300091E090939B08809368040895DA01A901C6
:1022400090E026E130E0829FF001839FF00D929FA5
:10225000F00D1124E456F74F618710861286B18382
:10226000A0831282138255834483168217820895B5
:1022700090E026E130E0829FD001839FB00D929FD5
:10228000B00D1124A456B74F6623D1F412968C9149
:10229000129790E0880F991FED91FC911197E80F2C
:1022A000F91F5183408312968C9112978F5F12967B
:1022B0008C9312978430F1F412961C921297089521
:1022C00016968C91169790E0880F991F1496ED91B1
:1022D000FC911597E80FF91F5183408316968C9156
:1022E00016978F5F16968C931697843019F416966E
:1022F0001C9216970895CF93DF93EA0190E026E1B0
:1023000030E0829FD001839FB00D929FB00D1124C9
:10231000A456B74F662309F513968C91139712961E
:102320009C9112978917D9F190E0880F991FED9130
:10233000FC911197E80FF91F80819181998388831F
:1023400013968C9113978F5F13968C931397843009
:1023500041F513961C92139724C017968C911797EA
:1023600016969C9116978917D1F090E0880F991FC7
:102370001496ED91FC911597E80FF91F80819181DA
:102380009983888317968C9117978F5F17968C93F4
:102390001797843031F417961C92179702C081E08A
:1023A00001C080E0DF91CF910895EF92FF920F93EB
:1023B0001F93CF93DF9300D0CDB7DEB7F82E282F31
:1023C00030E086E190E0289F8001299F100D389F22
:1023D000100D11240456174FF8018085882309F049
:1023E000BCC08285813041F0813068F0823089F054
:1023F000833009F04BC028C025B1F8019185909534
:10240000922395B942C085B1F8019185892B85B990
:102410003BC0F8018585882349F095B18185809579
:10242000892385B98585815085870BC0F80186850C
:10243000882339F085B19185892B85B986858150AE
:102440008687F80186851AC0F8018685882341F0C1
:1024500085B19185892B85B98685815086870CC089
:10246000F8018585882341F095B181858095892380
:1024700085B9858581508587F8018585882331F464
:10248000838585878485868781E08787F801E7844F
:10249000F1E0EF1609F0CEC08F2D61E0AE014F5F85
:1024A0005F4F0E947B11882321F5F801E086498166
:1024B0005A81CA019070009711F4108A4BC09C0198
:1024C000215030402A3F310540F482E0F801808BF2
:1024D000518B428B538B448B3DC08C3F910519F43B
:1024E000F801108637C08F3F9105A1F5F801E08A09
:1024F00031C08F2D60E0AE014F5F5F4F0E947B11B6
:10250000882341F589819A8190708130910551F03D
:102510008130910550F08230910551F08330910562
:10252000C9F40FC0F801E28615C0F801128612C086
:102530009AE0F80193878AE584879587868782E009
:1025400008C09AE5F80193878AE084879587868793
:1025500083E08287F80117866DC0F8018089813099
:1025600039F0813060F0823081F0833081F519C01C
:1025700025B1F80191859095922395B927C085B131
:10258000F8019185892B85B920C0F80184898823B9
:1025900041F085B19185892B85B984898150848BDF
:1025A0000CC0F8018389882341F095B1818580951D
:1025B000892385B983898150838BF8018389882396
:1025C00031F48189838B8289848B81E0858BF8014A
:1025D0008589882379F18F2D61E0AE014F5F5F4FD0
:1025E0000E947B11882321F561E0F8016087498111
:1025F0005A81CA019070009711F4108A19C09C0189
:10260000215030402A3F310540F482E0F801808BB0
:10261000518B428B538B448B0BC08C3F910519F42B
:10262000F801108605C08F3F910511F4F801608B09
:10263000F801158A0F900F90DF91CF911F910F91A4
:10264000FF90EF900895DB0190E026E130E0829F5B
:10265000F001839FF00D929FF00D1124E456F74F87
:1026600080858C93828511968C9311978485129620
:102670008C931297838513968C9313978089149665
:102680008C931497828915968C9315978189169649
:102690008C9316970895CF92DF92EF92FF920F934B
:1026A0001F93CF93DF930F92CDB7DEB77B01898362
:1026B0000E94632A898181600E94862A882321F4EE
:1026C0000E947B2A81E012C081E00E94BB2A182F61
:1026D00000E080E00E94BB2AC82EDD24C02AD12A57
:1026E0000E947B2AF701D182C08280E00F90DF91A7
:1026F000CF911F910F91FF90EF90DF90CF900895B1
:102700001F920F920FB60F920BB60F9211242F93B8
:102710003F934F935F936F937F938F939F93AF9369
:10272000BF93EF93FF930E94EB2A8091E103909176
:10273000E203A091E303B091E4030196A11DB11D52
:102740008093E1039093E203A093E303B093E40347
:102750008091E5039091E60301969093E6038093C0
:10276000E50323E0883E920739F481E08093E10895
:102770001092E6031092E5038091E7038F5F809348
:10278000E703843629F481E08093E2081092E7039E
:102790008091E8038F5F8093E8038A3071F40E9490
:1027A000622B81E08093EE081092E803809103048D
:1027B000882319F0815080930304FF91EF91BF911A
:1027C000AF919F918F917F916F915F914F913F91C9
:1027D0002F910F900BBE0F900FBE0F901F9018956A
:1027E00085B1817F85B9209A28988FEC97E0019771
:1027F000F1F700C0000021E0199B20E081E01A9B66
:1028000080E091E01B9B90E0289AEFECF7E0319795
:10281000F1F700C0000063B141E01A9B40E031E0F5
:102820001B9B30E051E061FF50E0251322E0841350
:1028300082E0931392E0E82FEE0FE80FE20F89E0B9
:10284000989F902D1124E90FF0E0E15BFA4F8491FD
:10285000089590E08057904062E070E00E949C2FC5
:10286000862F0895FC018481869586958170089550
:10287000FC0183819481890F819585838281DF01A9
:1028800023E090E005C015963C911597930F2F5FBC
:1028900011962817C0F3DF01A80FB11D919513966B
:1028A0009C9313978F5F82830895CF93DF93EC01FE
:1028B00088818E7F806888830E94F60F88818F7759
:1028C000888380E0DF91CF910895FC01838194811A
:1028D000890F819595819817D9F4828190E00197AD
:1028E00053E040E008C02E0F3F1FD90113962C91F2
:1028F0001397420F5F5F252F30E0281739079CF3AD
:10290000E80FF91F41958381841721F082E0089533
:1029100081E0089580E008959F92AF92BF92CF9298
:10292000DF92EF92FF920F931F93CF93DF93CDB778
:10293000DEB760970FB6F894DEBF0FBECDBF8C0137
:102940007B01FE013296ACE5B3E086E00D9001928A
:102950008150E1F7D80114962C911497269526956D
:102960002A3009F447C32B3040F4243009F44FC017
:10297000263011F00C94002009C02C3209F48FC4C9
:10298000203311F00C9400200C94471DF801808531
:10299000813011F00C9400208BED97E00E942C2CDC
:1029A000D80116968C911697F701838317969C9100
:1029B000179714968C9114978C5F8C7F292F237016
:1029C000822B84838091EC08868314968C911497D3
:1029D00083709C7F892B878318968C9118978087AA
:1029E0001186128681E8838782E0848783E7858762
:1029F00081E586878BE287878DEB808B82E9818BEF
:102A0000128A138A83E8848B82E10C943F20D801D8
:102A100018968C911897803209F49FC0813248F43F
:102A2000813009F446C0813088F0823009F0D9C283
:102A30006EC0823209F45EC1823208F4BDC08732B2
:102A400009F41AC28D3209F0CCC284C18FEF97E02D
:102A50000E942C2CF8018185809337098285809310
:102A600038098681D70113968C93139797818481B7
:102A70008C5F8C7F292F2370822B14968C93149754
:102A80008091EC0816968C931697848183709C7FB6
:102A9000892B17968C931797808518968C93189787
:102AA00019961C920E94F50A0E94902087E00C94CF
:102AB000191F8FE298E00E942C2CD80116968C9159
:102AC0001697F701838317969C91179714968C910C
:102AD00014978C5F8C7F292F2370822B84838091A5
:102AE000EC08868314968C91149783709C7F892BB5
:102AF000878318968C911897808711868091370963
:102B0000828780913809838789E00C943F208FE584
:102B100098E00E942C2CD80116968C911697F701FC
:102B2000838317969C91179714968C9114978C5FBA
:102B30008C7F292F2370822B84838091EC088683DD
:102B400014968C91149783709C7F892B8783189699
:102B50008C91189780871186FBC28BE898E00E94C1
:102B60002C2CD80116968C911697F7018383179613
:102B70009C91179714968C9114978C5F8C7F292FBA
:102B80002370822B84838091EC08868314968C9129
:102B9000149783709C7F892B878318968C918087EC
:102BA00011860E944B2AD7011A968C931A9781E0BE
:102BB0001B968C931B97CCC08CEB98E00E942C2C1E
:102BC000F8018681D70113968C931397978184819E
:102BD0008C5F8C7F292F2370822B14968C931497F3
:102BE0008091EC0816968C931697848183709C7F55
:102BF000892B17968C931797808518968C93189726
:102C000019961C92A384BB24948580E0A82AB92A33
:102C1000C58496840E944B2A0197A816B90629F408
:102C20008FEFF7018287838708C0C5010196D7011E
:102C30001A968C931A971B969C93F501EE0FFF1F23
:102C4000EE59FC4F0C2D10E060817181600F711FF7
:102C5000C7010C96492D50E00E94C32FB5E0BC156A
:102C600060F0C801890D911D8530910534F0F701A0
:102C7000E01BF10B8091EC08818BE2E0AE16B10411
:102C8000C8F4FDE0FC1570F1DD24C601890D911D2D
:102C90008D3091053CF1F701EC19FD098091EC08AC
:102CA00090E08057904062E070E00E949C2F605A54
:102CB000618F18C049E04C15A8F0DD24C601890DCC
:102CC000911D8930910574F0F701EC19FD0980918F
:102CD000EC0890E08057904062E070E00E949C2FEA
:102CE000605A658B892D875FD70112968C93129756
:102CF0000C94232088EE98E00E942C2CF801868109
:102D0000D70113968C931397978184818C5F8C7F66
:102D1000292F2370822B14968C9314978091EC08A2
:102D200016968C931697848183709C7F892B1796B7
:102D30008C931797808518968C93189719961C92E8
:102D4000199781E01A968C931A971B961C921B97E1
:102D500089E0CBCF88E199E00E942C2CF801868194
:102D6000D70113968C931397978184818C5F8C7F06
:102D7000292F2370822B14968C9314978091EC0842
:102D800016968C931697848183709C7F892B179657
:102D90008C931797808518968C93189719961C9288
:102DA000199781859AE012969C9312978430C9F105
:102DB000853058F4813009F1813098F0823001F18A
:102DC000833011F00C9423201EC0863009F43FC0DC
:102DD0008630D8F18730E9F1883011F00C94232047
:102DE00048C0F701128680EC83870E94D60AD7017B
:102DF0001C968C931C970C9423208091DF080AC0AA
:102E00008091E50815C080E00E9407099695879596
:102E100096958795F701828780E4838714860C94C2
:102E2000232081E00E9407099695879596958795BE
:102E3000D7011A968C931A9780E41B968C931B9754
:102E40001C961C921C970C94232082E0DDCF83E01B
:102E5000E9CFF701128680EC83870E947F20D7019B
:102E60001C968C930E947F20F70195878BE00C9431
:102E70003F208091F008DCCF88E499E00E942C2C60
:102E8000F8018681D70113968C93139797818481DB
:102E90008C5F8C7F292F2370822B14968C93149730
:102EA0008091EC0816968C931697848183709C7F92
:102EB000892B17968C931797808518968C93189763
:102EC00019961C9219978185843009F43CC085308D
:102ED00050F48130B9F0813090F08230E9F08330E5
:102EE00009F07DC026C0863009F441C08630A8F1C3
:102EF000873009F474C0883009F071C042C0F7010E
:102F00000C943D208FE3D7011A968C931A978091E9
:102F100068039091690309C08FE3D7011A968C93D7
:102F20001A9780916A0390916B03FC01B996E49122
:102F300033C08FE3D7011A968C931A9780916C0354
:102F400090916D03F2CF8FE3D7011A968C931A9765
:102F500080916E0390916F03E8CF8FE3D7011A96AB
:102F60008C931A978091700390917103DECF8FE359
:102F7000D7011A968C931A978091720390917303DC
:102F8000D4CF8FE3F7018287809176039091770306
:102F9000FC01B996E491D7011B96EC931B97FC01B9
:102FA000B896E4911C96EC931C97FC01B796E491BB
:102FB0001D96EC931D97FC01B696E4911E96EC933A
:102FC0001E97FC01B596E4911F96EC931F9784968B
:102FD000FC01849150968C9350978EE086CED70159
:102FE0001EC48BE799E00E942C2CF80180850E947A
:102FF000A52C48C5D80118968C911897813109F4F1
:1030000052C0823109F4B2C0803109F0F9C78DE9AC
:1030100099E0288B0E942C2CF8018185288988232F
:1030200051F08130D1F4288B0E947C20288988239C
:1030300011F483ED13C0D7011A961C921A9782E0FF
:103040001B968C931B971C961C921C9719961C928E
:10305000199712962C93129705C089ECF701818776
:1030600087E08283D80116968C911697F7018383A7
:1030700017969C91179714968C9114978C5F8C7F60
:10308000292F2370822B84838091EC0886831496E9
:103090008C91149783709C7F892B878318968C91D1
:1030A00018978087D0C78DEC99E00E942C2CD8010E
:1030B00016968C911697F701838317969C91179714
:1030C00014968C9114978C5F8C7F292F2370822B00
:1030D00084838091EC08868314968C911497837076
:1030E0009C7F892B878318968C91189780871186EF
:1030F0001A96AC901A97BB241B969C911B9780E064
:10310000A82AB92A1C96CC901C97C28619968C9135
:103110001997882321F0813009F095C70EC086EFFA
:1031200099E00E942C2CB50160507040C7010B96AD
:103130004C2D50E00E94E22F16C08BEF99E00E94C8
:103140002C2C0E947C20882329F483EDF7018187B1
:1031500087E095C79701255F3F4F80E5B5014C2D6E
:1031600050E00E94A0228C2D885FBECD80E09AE0C6
:103170000E942C2CF801C280F6EFCF0ED8011A96CF
:10318000AC901A97BB241B969C911B9780E0A82AB1
:10319000B92A19968C911997882321F0813009F06A
:1031A0005DC014C08AE29AE00E942C2CF701C2860E
:1031B000B50160507040C8010C964C2D50E00E9443
:1031C000FA2FD70119961C92199748C08FE29AE0FE
:1031D0000E942C2C8EE493E00E941A2CC5010E94C0
:1031E0005C2C84E593E00E941A2C8C2D90E00E94C8
:1031F0005C2C8CE493E00E941A2C0E947C20F70146
:10320000882349F1C28611868CE7BE016F5F7F4F2C
:103210000E9406218823B1F4698161616F77698317
:103220008CE70E942B21882311F0F70114C098012C
:10323000245F3F4F80E5B5014C2D50E00E943025C2
:10324000882361F0D7011A961C921A9783ED19967C
:103250008C93199703C0128683ED8187D801169647
:103260008C911697F701838317969C911797149664
:103270008C9114978C5F8C7F292F2370822B8483F1
:103280008091EC08868314968C91149783709C7FB0
:10329000892B878318968C9118978087EFC6D80161
:1032A00018968C9118978C3009F468C38D30A8F467
:1032B000853009F4B7C0863030F4882321F184309A
:1032C00009F0C8C357C0873009F4E2C0873008F45A
:1032D000DCC0883009F0BEC361C1893109F415C36F
:1032E0008A3138F48D3009F4C3C2813109F0B2C398
:1032F00075C38E3109F406C38D3209F43CC38A319B
:1033000009F0A8C335C384E39AE00E942C2CF8018D
:103310008681D70113968C931397978184818C5F54
:103320008C7F292F2370822B14968C931497809175
:10333000EC0816968C931697848183709C7F892B5A
:1033400017968C931797808518968C9318971996D3
:103350001C9219971A961C921A9782E31B968C93CB
:103360001B9781E01C968C931C971D961C921D97B1
:103370008BE0BBCC8CE59AE00E942C2CF801868176
:10338000D70113968C931397978184818C5F8C7FE0
:10339000292F2370822B14968C9314978091EC081C
:1033A00016968C931697848183709C7F892B179631
:1033B0008C931797808518968C93189719961C9262
:1033C00019971A961C921A9788E012968C93129766
:1033D0008285882321F0813009F04CC615C081E830
:1033E0009AE00E942C2CF8018385882321F08430F8
:1033F00009F040C606C01092EB0882E30E94312B10
:1034000022C60E94ED0A1FC686E89AE00E942C2C74
:10341000D8011B968C911B97843009F02BC60E9413
:103420008C2011C68BE89AE00E942C2CF801868132
:10343000D70113968C931397978184818C5F8C7F2F
:10344000292F2370822B14968C9314978091EC086B
:1034500016968C931697848183709C7F892B179680
:103460008C931797808518968C93189719961C92B1
:1034700019971A961C921A9787E01B968C931B97A4
:103480001C961C921C978AE030CC85EB9AE0B6C55E
:1034900081EE9AE00E942C2CF801248545858285D6
:1034A000882321F0813009F041C227C0C22EDD24DB
:1034B000942F80E0C82AD92A83858130B1F08130E9
:1034C00020F0823009F087C112C080E061E0A601DF
:1034D0000E9438110E94D30A823009F027C2CC2002
:1034E00009F024C20E94D90A21C281E001C082E011
:1034F00061E0A6010E94381119C2F801838581306C
:1035000081F0813018F0823049F516C0222319F07D
:103510002F3F29F402C080E015C080E01AC080E08F
:103520001BC0222319F02F3F29F402C081E00AC0FA
:1035300081E00FC081E010C0222319F02F3F59F421
:1035400007C082E060E040E020E00E944920EEC138
:1035500082E061E0F8CF82E062E0F7CFD8018681B7
:10356000F701838317969C91179714968C91149763
:103570008C5F8C7F292F2370822B84838091EC08B1
:10358000868314968C91149783709C7F892B8783F4
:1035900018968C91189780878CEC6EC58BE09BE019
:1035A0000E942C2C19820DC0F801E80FF11D8381B7
:1035B0000E94A52C8AE593E00E941A2C89818F5FD6
:1035C00089838981D80112969C911297891760F39B
:1035D0008CE493E00E941A2CF8018285882309F07C
:1035E00023C18385813009F44FC0813020F08230BF
:1035F00009F0E4C08FC080E0BE01685F7F4F0E9489
:1036000023138985882319F0813071F404C0F701F0
:10361000148615860EC08FEFD7011C968C931C97CD
:103620001D961C921D9705C08A85F70184878B859E
:10363000858781E0D7011E968C931E979CE0129699
:103640009C9312979885913009F0B5C082E01B9643
:103650008C931B978C85882319F0813071F404C0FA
:10366000F7011786108A0EC08FEFD7011F968C9333
:103670001F9750961C92509705C08D85F70187873C
:103680008E85808B81E08DC081E0BE01685F7F4FB9
:103690000E9423138985882319F0813071F408C0B2
:1036A000D7011C961C921C971D961C921D970EC04C
:1036B0008FEFF7018487158609C08A85D7011C968C
:1036C0008C931C978B851D968C931D9782E0F70138
:1036D00086879CE0928398859130C9F483878C8596
:1036E000882319F0813049F403C01786108A09C075
:1036F0008FEFF7018787108A04C08D8587878E85B5
:10370000808B82E0F701818B8FE082838DC081E026
:1037100083878AC082E0BE01685F7F4F0E942313C7
:103720008985882319F0813071F404C0F70114866B
:1037300015860EC08FEFD7011C968C931C971D9693
:103740001C921D9705C08A85F70184878B85858724
:1037500083E0D7011E968C931E978CE012968C9373
:1037600012978885813031F582E01B968C931B97E8
:103770008C85882319F0813071F404C0F701178615
:10378000108A0EC08FEFD7011F968C931F9750960B
:103790001C92509705C08D85F70187878E85808B99
:1037A00083E0D70151968C9351978FE012968C93BA
:1037B00012973AC081E0F701838736C085E39BE02A
:1037C0000E942C2CD8011A968C910E94A52C83E67D
:1037D0009BE00E942C2CF8018681D70113968C93D4
:1037E0001397978184818C5F8C7F292F2370822B84
:1037F00014968C9314978091EC0816968C931697D8
:10380000848183709C7F892B17968C931797808572
:1038100018968C9318978CEC19968C9319971A9686
:103820001C921A9788E061CAF8018681D701139625
:103830008C931397978184818C5F8C7F292F2370C1
:10384000822B14968C9314978091EC0816968C9387
:103850001697848183709C7F892B17968C9317977A
:10386000808518968C93189719961C92199746C0C4
:1038700085E69BE00E942C2CF8018285882319F0B4
:103880008130A1F40CC0D7011B961C921B971C968B
:103890001C921C9719961C9219978AE00DC0F7018B
:1038A0008387148611868AE0828308C08CECD70156
:1038B00019968C93199787E012968C93F80186815C
:1038C000D70113968C931397978184818C5F8C7F9B
:1038D000292F2370822B14968C9314978091EC08D7
:1038E00016968C931697848183709C7F892B1796EC
:1038F0008C931797808518968C9318971A961C921C
:103900001A97A1C382E99BE079C38CEB9BE00E94EC
:103910002C2CF8018685882319F00E94DD0A06C048
:103920000E94D30A853011F40E94E50AD801169648
:103930008C911697F701838317969C91179714968D
:103940008C9114978C5F8C7F292F2370822B84831A
:103950008091EC08868314968C91149783709C7FD9
:10396000892B878318968C9118978087118685C339
:1039700087EE9BE043C382E19CE040C38AE39CE086
:103980000E942C2CD80116968C911697F7018383F0
:1039900017969C91179714968C9114978C5F8C7F37
:1039A000292F2370822B84838091EC0886831496C0
:1039B0008C91149783709C7F892B878318968C91A8
:1039C00018978087128688E082831A968C911A97BE
:1039D0008823A1F1813009F036C3B7C185E69CE0A8
:1039E0000E942C2CD80116968C911697F701838390
:1039F00017969C91179714968C9114978C5F8C7FD7
:103A0000292F2370822B84838091EC08868314965F
:103A10008C91149783709C7F892B878318968C9147
:103A200018978087128688E082831A968C911A975D
:103A3000882321F0813009F006C302C08FEF18C13E
:103A4000F8018385882319F00E948420CDC20E944A
:103A50008820CAC28DE89CE00E942C2C19820DC0DF
:103A6000F801E80FF11D83810E94A52C8AE593E0FF
:103A70000E941A2C89818F5F89838981F801928144
:103A8000891770F38CE493E00E941A2CB9C2D80114
:103A900018962C911897243009F40EC1253060F443
:103AA0002130E9F0213008F485C1223009F468C0E2
:103AB000233009F0A1C2B2C0273009F4F1C1283087
:103AC00038F4253009F444C1263009F095C2B3C159
:103AD000283009F424C2293009F08EC256C289EA7E
:103AE0009CE00E942C2CF801C1849284D384A4848D
:103AF0008681D70113968C931397978184818C5F6D
:103B00008C7F292F2370822B14968C93149780918D
:103B1000EC0816968C931697848183709C7F892B72
:103B200017968C931797808518968C93189787E033
:103B300012968C93B0E1BA1510F482E85BC20E9431
:103B40007C20882309F493C0CC2011F490E5C92E81
:103B5000692D70E09D2D80E0682B792B9701265F01
:103B60003F4F8C2D4A2D50E00E94A022882309F05F
:103B7000A1C0D70119961C9219978A2D895FB5C8E3
:103B80008EEC9CE00E942C2CF801C184A284D3848A
:103B900044858681D70113968C93139797818481EE
:103BA0008C5F8C7F292F2370822B14968C93149713
:103BB0008091EC0816968C931697848183709C7F75
:103BC000892B17968C931797808518968C93189746
:103BD00087E012968C931297413110F082E849C029
:103BE000488B0E947C204889882311F480E802C217
:103BF000CC2011F480E5C82E6A2D70E09D2D80E068
:103C0000682B792B9801235F3F4F8C2D50E00E9449
:103C10003025882309F499C081E82AC084EF9CE00C
:103C20000E942C2CD80116968C911697F70183834D
:103C300017969C91179714968C9114978C5F8C7F94
:103C4000292F2370822B84838091EC08868314961D
:103C50008C91149783709C7F892B878318968C9105
:103C6000808787E082830E947C20882331F480E86B
:103C7000D70119968C931997E6C18CE7BE016F5F47
:103C80007F4F0E9406218823A9F48981982F916192
:103C9000D80119962C911997222311F0816902C03D
:103CA000892F8F7789838CE769810E942B21882354
:103CB00009F49AC181E89EC18EE19DE00E942C2CFE
:103CC000F8018681D70113968C931397978184818D
:103CD0008C5F8C7F292F2370822B14968C931497E2
:103CE0008091EC0816968C931697848183709C7F44
:103CF000892B17968C931797808518968C93189715
:103D000087E012968C93129782B18C7F82B981855D
:103D100080FD119AF801818581FD109A8FEF9FE057
:103D20000E94F22F8983D80119966C91199790E01F
:103D3000262F30E08227932783709070009729F018
:103D400063708FEF9FE00E940430F70111867BC102
:103D50008AE49DE00E942C2CD80116968C9116972F
:103D6000F701838317969C91179714968C9114975B
:103D70008C5F8C7F292F2370822B84838091EC08A9
:103D8000868314968C91149783709C7F892B8783EC
:103D900018968C911897808787E08283389A8FEFE6
:103DA00099E6A8E181509040A040E1F700C00000F2
:103DB00038981AC18EE69DE00E942C2CF80186816D
:103DC000D70113968C931397978184818C5F8C7F96
:103DD000292F2370822B14968C9314978091EC08D2
:103DE00016968C931697848183709C7F892B1796E7
:103DF0008C931797808518968C93189787E0129666
:103E00008C93129719961C92199720E00FC0822F5D
:103E100090E0F701E80FF91F42E050E04C0F5D1F02
:103E2000840F951FDC018C9182872F5F253078F3FA
:103E30008CE0F70124C189E99DE00E942C2CD80177
:103E400016968C911697F701838317969C91179776
:103E500014968C9114978C5F8C7F292F2370822B62
:103E600084838091EC08868314968C9114978370D8
:103E70009C7F892B878318968C911897808787E081
:103E800082838DEC81878091E903882309F4DBC06C
:103E9000A701465F5F4F8CE061E00E940D296AC078
:103EA00085EC9DE0288B0E942C2CD80119968C91D2
:103EB0001997809341091A968C911A978093420919
:103EC00016968C911697F701838317969C911797F6
:103ED00014968C9114978C5F8C7F392F3370832BC1
:103EE00084838091EC08868314968C911497837058
:103EF0009C7F892B878318968C91189780872889B7
:103F000022838DEC81878091E903882309F49BC08B
:103F10008CE061E041E459E00E94F52563C081EF47
:103F20009DE00E942C2CD80116968C911697F701D3
:103F3000838317969C91179714968C9114978C5F96
:103F40008C7F292F2370822B84838091EC088683B9
:103F500014968C91149783709C7F892B8783189675
:103F60008C91808787E08283B7016F5E7F4F88E402
:103F70000E946F298823E9F5D70112968C91129738
:103F80008E5F12968C93129730C08EE19EE00E9455
:103F90002C2CD80119966C911997609341091696AB
:103FA0008C911697F701838317969C911797149617
:103FB0008C9114978C5F8C7F292F2370822B8483A4
:103FC0008091EC08868314968C91149783709C7F63
:103FD000892B878318968C91808787E0828388E479
:103FE0000E944829882329F4D70119961C92199711
:103FF0002AC08FEFF70126C089E49EE00E942C2C96
:10400000D80116968C911697F701838317969C9189
:10401000179714968C9114978C5F8C7F292F23709F
:10402000822B84838091EC08868314968C9114975C
:1040300083709C7F892B878318968C91808787E07B
:10404000828381EC8187D70111961C92119781E0C0
:1040500060960FB6F894DEBF0FBECDBFDF91CF9153
:104060001F910F91FF90EF90DF90CF90BF90AF9096
:104070009F9008958CECF7018187128688E08283F7
:10408000E2CF83EF98E00895FC01878186958695BD
:104090000895982F842F913099F0913018F0923034
:1040A00051F51CC060933A093AE0632F0E94902FAB
:1040B00080934009822F0E94902F80933C0908959D
:1040C00060933F093AE0632F0E94902F8093450947
:1040D000822F0E94902F80933E09089560933909A2
:1040E0003AE0632F0E94902F80934409822F0E9410
:1040F000902F8093560908958091B7030895809179
:10410000F0039091F103089581E08093EF03089507
:1041100081E08093EE03089581E08093ED0308959C
:1041200081E08093EB0308951F93CF93DF93CDB786
:10413000DEB7C354D0400FB6F894DEBF0FBECDBF7C
:10414000182F80ED90E10E942C2C812F0E94A52C2D
:1041500088E793E00E941A2C809137098C8380E1D4
:104160008D838091EC088F838091360988878C5FDE
:104170008093360982E0898784E08A8782EF8B8783
:1041800087E08C878FE68D871E878BE08B83CE013F
:1041900001960E94381481E08A83CE0101960E9424
:1041A000FA101093B503CD5BDF4F0FB6F894DEBF66
:1041B0000FBECDBFDF91CF911F91089580913B0934
:1041C000982F917080FD08C08091FC03882321F016
:1041D0001092FC0381E008959093FC0380E0089521
:1041E00080913B09982F917080FF08C08091FD035A
:1041F000813021F081E08093FD0308959093FD03C9
:1042000080E0089590913B09892308950F931F93AF
:10421000CF93DF930F92CDB7DEB78B0189830E94D6
:10422000C029898181600E94E329882321F40E94AA
:10423000D82981E00AC080E00E94192A89830E945F
:10424000D8298981F801808380E00F90DF91CF9198
:104250001F910F9108951F93CF93DF9300D0CDB797
:10426000DEB76A8389830E94C02989810E94E3297D
:104270006A81882321F40E94D82981E009C0862F11
:104280000E94E329182F0E94D82981E0111180E0B3
:104290000F900F90DF91CF911F9108951F93CF93AF
:1042A000DF930F92CDB7DEB780913A09813029F0C4
:1042B0008130E0F08230F1F405C01092F4031092E6
:1042C000F50309C08091F40390914009891728F4FF
:1042D0008F5F8093F40311E00EC08091F5038F5F30
:1042E0008093F50390913C09891721F41092F4030F
:1042F0001092F50310E080913F09813029F0813060
:10430000F0F0823001F506C01092F6031092F70328
:10431000126019C012608091F603909145098917C7
:1043200020F48F5F8093F6030EC01D7F8091F7030A
:104330008F5F8093F70390913E09891721F41092C3
:10434000F6031092F70380913909813029F081300A
:10435000F0F0823001F506C01092F8031092F903D4
:10436000146019C014608091F80390914409891772
:1043700020F48F5F8093F8030EC01B7F8091F903B8
:104380008F5F8093F90390915609891721F4109259
:10439000F8031092F9038091B703882311F18CE799
:1043A000BE016F5F7F4F0E9406218823D1F481E018
:1043B0008093F203898180933B098F61898310FF89
:1043C00002C08D7F898311FF03C089818B7F898320
:1043D00012FF03C08981877F89838CE769810E94EE
:1043E0002B210F90DF91CF911F9108951F93CF93B1
:1043F000DF9300D0CDB7DEB7162F8CE7BE016F5F1D
:104400007F4F4A830E9406214A81882381F4642FCA
:1044100061236161409589814823642B69838CE71E
:104420000E942B2191E0882319F490E001C091E0D3
:10443000892F0F900F90DF91CF911F9108951F93B7
:10444000CF93DF930F92CDB7DEB789830E94C02947
:1044500089810E94E329882329F089E00E94E329C9
:10446000882321F40E94D82981E009C080E00E94BD
:10447000E329182F0E94D82981E0111180E00F90C4
:10448000DF91CF911F910895CF92DF92EF92FF922B
:104490000F931F93CF93DF930F92CDB7DEB7F82E14
:1044A0008B016A010E94C0298F2D0E94E329882375
:1044B00079F080E00E94E329882351F00E94CB2903
:1044C000EE24E394EF288E2D0E94E329882321F423
:1044D0000E94D82981E02AC080E00E94192A89839D
:1044E0000E94D8298981F80180830E94C0298F2DDC
:1044F0000E94E329882361F081E00E94E329882358
:1045000039F00E94CB298E2D0E94E329882321F4C3
:104510000E94D82982E00AC080E00E94192A89837B
:104520000E94D8298981F601808380E00F90DF9175
:10453000CF911F910F91FF90EF90DF90CF90089552
:10454000AF92BF92CF92DF92EF92FF920F931F93A1
:10455000CF93DF930F92CDB7DEB7182F062F6A01E6
:10456000E22EA32E79830E94C029812F880F0E94FA
:10457000E3297981882391F1872F0E94E3298823F9
:1045800069F1802F0E94E329882341F10E94CB2901
:10459000812F880F81600E94E3298823F9F00E2D76
:1045A0001A2DEE24FF2456010894A108B1080FC06B
:1045B000EA14FB0411F480E001C081E00E94192A92
:1045C000F80180830894E11CF11C0F5F1F4FEC146D
:1045D000FD0471F70E94D82980E003C00E94D82909
:1045E00081E00F90DF91CF911F910F91FF90EF909D
:1045F000DF90CF90BF90AF900895EF92FF920F930E
:104600001F93CF93DF93CDB7DEB728970FB6F894FB
:10461000DEBF0FBECDBF7C0180E560E070E048E00A
:1046200050E09E012F5F3F4F0E94A022882309F097
:1046300044C0FE01319697E02191820F9150E1F73D
:1046400081959885891731F08AE793E00E941A2CAA
:1046500082E034C00E8110E083E0000F111F8A95C4
:10466000E1F70115110539F180E5B80145E050E0A9
:104670009E012F5F3F4F0E94A0228823F1F42A81E0
:104680009981920F8B81980F3C81930F91953D8179
:10469000931731F080E993E00E941A2C84E00EC059
:1046A00090E00596080F191F27FFDECFF701118351
:1046B000008380E003C083E001C081E028960FB64C
:1046C000F894DEBF0FBECDBFDF91CF911F910F9148
:1046D000FF90EF9008959F92AF92BF92CF92DF929A
:1046E000EF92FF920F931F93CF93DF93CDB7DEB777
:1046F000C850D1400FB6F894DEBF0FBECDBF6C01DD
:10470000962E5A01FC01108280E560E070E048E0DE
:1047100050E09E012F5F3F4F0E94A022882309F0A6
:104720006DC0FE01319697E02191820F9150E1F723
:1047300081959885891709F05BC00E8110E093E0A0
:10474000000F111F9A95E1F70115110509F452C0E8
:1047500080E5B80145E050E09E012F5F3F4F0E9489
:10476000A022882309F04AC08A819981890FEB80B1
:104770008E0D9C81890F81959D818917E9F5FF2414
:104780000B5F1F4F80E5B801A7019E01275F3F4FD8
:104790000E94A022882391F590E00AC049E050E0F1
:1047A0004C0F5D1F240F351FF9012081920F8F5F81
:1047B000282F30E02E153F0588F391958C819817AE
:1047C000F9F4F60180818F5F8083891559F4A11473
:1047D000B10441F0F501DE0119968DE00D900192D2
:1047E0008150E1F78A8187FD0DC00E0D1F1DB0CFEE
:1047F00082E009C083E007C084E005C081E003C017
:1048000085E001C080E0C85FDE4F0FB6F894DEBFE0
:104810000FBECDBFDF91CF911F910F91FF90EF9011
:10482000DF90CF90BF90AF909F9008957F928F922E
:104830009F92AF92BF92CF92DF92EF92FF920F932F
:104840001F93CF93DF93CDB7DEB7A1970FB6F89440
:10485000DEBF0FBECDBF85E78B8384E48C8387E505
:104860008D8383E48E831092E90332E0E32EF12CF2
:10487000EC0EFD1EC70160E040E050E00E94F90A26
:104880005E010894A11CB11CC50160E040E050E04D
:104890000E946B238A81882319F489E890E106C07D
:1048A0008981882309F07DC082EA90E10E942C2C46
:1048B00011E08CC0872D982D6D2DAE014C5E5F4FA1
:1048C0000E94F90A8BEB90E10E942C2C8E010C5E69
:1048D0001F4F20E0F80181918F0129A30E94A52C90
:1048E0008DEA93E00E941A2C29A12F5F2D3091F7B9
:1048F00088E793E00E941A2C11E001E0AA24A39417
:104900004AC0892D9C2D602FAE01495F5F4F0E94E8
:104910006B238A85803351F5112341F186EC90E1B8
:104920000E942C2C27E0E22EF12CEC0EFD1E10E054
:10493000F70181917F010E94A52C8DEA93E00E94EE
:104940001A2C1F5F1D30A1F788E793E00E941A2CF4
:10495000CE014796BE01665F7F4F4AE050E00E945D
:10496000CC2F009711F011E001C010E08A8582334E
:1049700089F48091E903882369F4CE010396BE018E
:10498000645F7F4F44E050E00E94CC2F009711F409
:10499000A092E9030F5F8981801708F0B2CFD3940A
:1049A00007C011E0DD24D3947E2C8F2C9A2CCB2CC5
:1049B0008A818D1518F0112309F07CCF91E0111137
:1049C00090E08091E90389238093E903812FA196E8
:1049D0000FB6F894DEBF0FBECDBFDF91CF911F9110
:1049E0000F91FF90EF90DF90CF90BF90AF909F908E
:1049F0008F907F9008950F931F93CF93DF9300D0F4
:104A0000CDB7DEB7062F142F7A8389830E94C02981
:104A10008981880F0E94E3297A81882351F0872FAA
:104A20000E94E329882329F0802F0E94E32988230C
:104A300021F40E94D82981E00CC0812F0E94E32933
:104A40000E94D8298FE097E20197F1F700C000009B
:104A500080E00F900F90DF91CF911F910F910895FB
:104A6000AF92BF92CF92DF92EF92FF921F93CF93BC
:104A7000DF93182F6B015A017901C0E0D0E00AC022
:104A8000F70141917F01BE016C0D7D1D812F0E94B8
:104A9000FB242196CA15DB0599F780E0DF91CF91C1
:104AA0001F91FF90EF90DF90CF90BF90AF9008954F
:104AB000AF92BF92CF92DF92EF92FF920F931F932C
:104AC000CF93DF930F92CDB7DEB7082F6A01E22EA6
:104AD000A32E69830E94C029802F880F0E94E3299A
:104AE00069818823B9F0862F0E94E329882391F0F9
:104AF0000E94CB29802F880F81600E94E3298823A0
:104B000049F00E2D1A2DEE24FF2456010894A10819
:104B1000B10813C00E94D82981E015C0EA14FB0433
:104B200011F480E001C081E00E94192AF80180831D
:104B30000894E11CF11C0F5F1F4FEC14FD0471F78A
:104B40000E94D82980E00F90DF91CF911F910F91A3
:104B5000FF90EF90DF90CF90BF90AF900895CF92ED
:104B6000DF92EF92FF920F931F93CF93DF9300D0CA
:104B7000CDB7DEB77A0169016A8389830E94C029B3
:104B80008981880F0E94E3296A81882381F0862F1A
:104B90000E94E329882359F08601CC24DD240EC02D
:104BA000F80181918F010E94E329882321F40E945A
:104BB000D82981E00FC00894C11CD11CCE14DF0499
:104BC00079F70E94D8298FE097E20197F1F700C0AA
:104BD000000080E00F900F90DF91CF911F910F9117
:104BE000FF90EF90DF90CF9008950F931F93CF9396
:104BF000DF9300D0CDB7DEB78A016A8389830E9434
:104C0000C0298981880F0E94E3296A818823E1F005
:104C1000862F83700E94E3298823B1F0F8018081F8
:104C20000E94E329882381F0F80181810E94E32911
:104C3000882351F00E94D8298FE097E20197F1F77D
:104C400000C0000080E003C00E94D82981E00F90DE
:104C50000F90DF91CF911F910F910895CF92DF9226
:104C6000EF92FF928091B7038093B6032091F303F4
:104C70002093B7038091F203882389F030913B0998
:104C80008091F0039091F10330FD03C08D7F81602E
:104C900002C082608E7F9093F1038093F0032330F3
:104CA00009F467C1243048F48091B603213009F437
:104CB000A1C0223008F023C10DC0253009F4E7C19E
:104CC000253008F460C1263009F42DC22B3009F0DC
:104CD00057C264C0882389F180E490E09093F10387
:104CE0008093F003469883E69EE00E942C2C80E798
:104CF0009EE00E942C2C8091F1030E94A52C8091B3
:104D0000F0030E94A52C88E793E00E941A2C0E94D1
:104D1000592A1092FA0380E060E040E020E00E940F
:104D2000492081E060E040E020E00E94492082E0EC
:104D300060E040E020E00E9449201092F2033599A3
:104D40002AC00E94662B882329F08091FA038F5F86
:104D50008093FA038091FA03843608F411C20E940A
:104D6000AA29882321F48BE79EE00E942C2C109224
:104D7000FA038091F0039091F1038F7B806290930E
:104D8000F1038093F00380E061E040E020E00E94C6
:104D900049208BE0F3C11092FA03F2C18091E3083D
:104DA000882309F4EDC18EE99EE00E942C2CC0906E
:104DB000E103D090E203E090E303F090E4030E946B
:104DC00016248093FB038091E1039091E2038C19F8
:104DD0009D090E945C2C89EB9EE00E942C2C0E9475
:104DE000552A85E00E94942081E08093F30380930C
:104DF000EA03C6C1813009F444C08DEB9EE00E94F5
:104E00002C2C8091B6038B3069F58091FB038823AD
:104E100099F48AEC9EE00E942C2C87E00E9494205A
:104E20008091F0039091F10380689093F103809357
:104E3000F00381E060E012C080EE9EE00E942C2C26
:104E400088E00E9494208091F0039091F10391609A
:104E50009093F1038093F00381E061E040E020E073
:104E60000E9449208FEF9EE00E942C2C8091F1033C
:104E70000E94A52C8091F0030E94A52C8AE09FE05F
:104E80007FC08091F00387FF35C08091E3088823BD
:104E900089F18091F203882361F00E94DE2088234B
:104EA00041F08CE09FE00E942C2C80E00E94942036
:104EB00015C08091F2038823A1F08091EA03882332
:104EC00081F080913B0980FD0CC086E29FE00E944A
:104ED0002C2C80E00E9494201092EA0382E08093C0
:104EE000F3038091EF03882329F084E08093F30398
:104EF0001092EF03359B44C184E49FE036C18230B9
:104F0000A1F089E59FE00E942C2C86E69FE00E949C
:104F10002C2C8091F1030E94A52C8091F0030E941B
:104F2000A52C88E793E00E941A2C0E94F020882389
:104F300051F081E79FE00E942C2C81E00E94942098
:104F400081E08093F303359B09C085E89FE00E94D0
:104F50002C2C86E00E9494201092F3038091EF03A2
:104F6000882309F40DC184E08093F3031092EF03CA
:104F700007C18091B603833009F402C18AE99FE03A
:104F80000E942C2CFDC08091B603843071F1809179
:104F9000F0039091F1038B7F9093F1038093F003E2
:104FA00087EA9FE00E942C2C84EB9FE00E942C2C2F
:104FB0008091F1030E94A52C8091F0030E94A52C02
:104FC00088E793E00E941A2C469A1092FA03809187
:104FD000E903882351F08CE061E043EB53E00E9449
:104FE000F5258FEB9FE00E942C2C0E94662B8823D6
:104FF00039F08091FA038F3118F48F5F8093FA03B0
:105000008091FA038E3159F48CE760E040E40E940D
:10501000F62182E061E040E020E00E9449200E9409
:10502000F0208823A1F08091F0039091F103826039
:105030008E7F9093F1038093F0038AED9FE00E94AE
:105040002C2C81E00E94942085E08093F3038091D2
:10505000ED03882319F085E08093F303359B90C01E
:105060008EEE9FE00E942C2C86E00E94942080917E
:10507000E903882309F47EC08CE061E04FEA53E045
:105080000E94F52583E090E10E942C2C73C0809152
:10509000B603853041F189E190E10E942C2C86E233
:1050A00090E10E942C2C8091F1030E94A52C80910C
:1050B000F0030E94A52C88E793E00E941A2C82E05E
:1050C00060E040E020E00E9449208091E9038823CD
:1050D00051F08CE061E04FEA53E00E94F52581E356
:1050E00090E10E942C2C8091ED03882371F0809137
:1050F000F0039091F10384609093F1038093F003A7
:1051000082E00E9494201092ED038091EE038823A8
:1051100029F086E08093F3031092EE03359B30C0B4
:1051200087E490E122C08091B6038630D1F08CE70D
:1051300060E440E40E94F62146988CE590E10E94EC
:105140002C2C89E690E10E942C2C8091F1030E9486
:10515000A52C8091F0030E94A52C88E793E00E9483
:105160001A2C359B0AC084E790E10E942C2C86E023
:105170000E9494201092F30303C081E08093F30314
:105180008091EB03882309F443C08091F00380FFF2
:1051900003C080E00E9494208091F00381FF03C04F
:1051A00081E00E9494208091F00382FF03C082E09E
:1051B0000E9494208091F00383FF03C083E00E944B
:1051C00094208091F00384FF03C084E00E94942027
:1051D0008091F00385FF03C085E00E9494208091B8
:1051E000F00386FF03C086E00E9494208091F003C4
:1051F00087FF03C087E00E9494208091F003909184
:10520000F10390FF03C088E00E9494201092EB030A
:10521000FF90EF90DF90CF900895EF92FF921F9351
:10522000CF93DF930F92CDB7DEB7182F7A01698342
:105230000E94C029812F880F0E94E3296981882359
:10524000E9F0862F83700E94E3298823B9F00E9439
:10525000CB29812F880F81600E94E329882371F078
:1052600081E00E94192AF701808380E00E94192AB8
:10527000F70181830E94D82980E003C00E94D829C9
:1052800081E00F90DF91CF911F91FF90EF900895F3
:10529000CF93DF9300D0CDB7DEB76A8389830E94B6
:1052A000C0298981880F0E94E3296A81882329F017
:1052B000862F0E94E329882321F40E94D82981E0C7
:1052C00009C00E94D8298FE097E20197F1F700C04A
:1052D000000080E00F900F90DF91CF910895CF9262
:1052E000DF92EF92FF920F931F93CF93DF930F9272
:1052F000CDB7DEB77B0189830E94C0298981880FE1
:1053000081600E94E329882321F40E94D8298FEF2D
:1053100017C081E00E94192A182F00E080E00E9447
:10532000192AC82EDD24C02AD12A0E94D829E114C6
:10533000F10411F48D2D04C0F701D182C08280E008
:105340000F90DF91CF911F910F91FF90EF90DF9021
:10535000CF9008958BB18F7C8BB98AB18F7C8AB93D
:1053600089E096E09A95F1F700C0549A96E09A95F4
:10537000F1F700C054988150A1F789B18072089567
:10538000559A86E08A95F1F700C0549A86E08A958E
:10539000F1F700C00895559886E08A95F1F700C0AE
:1053A000549886E08A95F1F700C00E94C0290895BC
:1053B000549886E08A95F1F700C0559886E08A9562
:1053C000F1F700C00895F89428E030E090E8492F04
:1053D000482311F4559A01C0559846E04A95F1F7D3
:1053E00000C054984DE04A95F1F70000549A46E009
:1053F0004A95F1F700C096952150304041F75598F5
:1054000086E08A95F1F700C0549846E04A95F1F796
:1054100000C099B186E08A95F1F700C0549A559A78
:1054200046E04A95F1F700C0789481E095FD80E070
:105430000895282FF894559898E080E0880F36E07A
:105440003A95F1F700C0549836E03A95F1F700C06C
:105450004D99816036E03A95F1F700C0549A36E0F4
:105460003A95F1F700C0915049F7222311F0559A6F
:1054700001C0559896E09A95F1F700C054983DE028
:105480003A95F1F70000549A559A96E09A95F1F7FB
:1054900000C0789408958091FE03882319F08BE072
:1054A00090E0089589E090E0089581E08093FE0304
:1054B00008951092FE0308958BB18F738BB98AB152
:1054C0008F738AB90895579A86E08A95F1F700C0DC
:1054D000569A86E08A95F1F700C00895579886E0BD
:1054E0008A95F1F700C0569886E08A95F1F700C0DA
:1054F0000E94632A0895569886E08A95F1F700C0C5
:10550000579886E08A95F1F700C0089528E030E0CA
:1055100090E8492F482311F4579A01C0579846E064
:105520004A95F1F700C056984DE04A95F1F7000012
:10553000569A46E04A95F1F700C0969521503040C2
:1055400041F7579886E08A95F1F700C0569896E0A3
:105550009A95F1F700C089B146E04A95F1F700C08D
:10556000569A579A96E09A95F1F700C08095881F51
:105570008827881F0895282F579898E080E0880F83
:1055800036E03A95F1F700C0569836E03A95F1F7D3
:1055900000C04F99816036E03A95F1F700C0569A05
:1055A00036E03A95F1F700C0915049F7222311F007
:1055B000579A01C0579896E09A95F1F700C056980F
:1055C0003DE03A95F1F70000569A579A96E09A9581
:1055D000F1F700C008959091590983B1809589270A
:1055E0009091FF03982390959093FF0320910004DE
:1055F0002823292720930004982392238091590976
:105600008927809359092091580980915909892344
:10561000822B8093580920915709809159098095D0
:105620008923822B809357090895F8949091580903
:105630008923909158099827909358097894089550
:10564000F89490915709892390915709982790933E
:10565000570978940895F89490915909789489237A
:1056600008958093050481E08093040408951092C6
:105670000404089581E090910404992309F480E0E2
:10568000089580910504882329F0815080930504B2
:1056900080E0089581E008958093030481E0809381
:1056A0000204089510920204089581E0909102048A
:1056B000992309F480E0089581E090910304911109
:1056C00080E0089581E080930104089580910104B1
:1056D000882321F01092010481E0089580E008956C
:1056E0001092C5008CE08093C40088E98093C100CB
:1056F0001092DC091092DA091092DB0910925D0A0F
:1057000008959091DA092091DC0991509F7729172B
:10571000C1F3E091DC09F0E0E352F64F8083809121
:10572000DC098F5F8093DC098091DC09803811F4FB
:105730001092DC098091C10080628093C1000895BD
:105740003091DB0920915D0A3217A1F020915D0AAA
:10575000E22FF0E0E65AF64F3081FC0130832F5FF4
:1057600020935D0A80915D0A803831F410925D0AC1
:1057700080E0089581E0089580E008951F920F92DF
:105780000FB60F920BB60F9211248F939F93EF9346
:10579000FF93E091DA09F0E0E352F64F80818093C5
:1057A000C6008091DA098F5F8093DA098091DA0967
:1057B000803811F41092DA099091DC098091DA09AD
:1057C000981729F48091C1008F7D8093C100FF91CB
:1057D000EF919F918F910F900BBE0F900FBE0F9086
:1057E0001F9018951F920F920FB60F920BB60F9243
:1057F00011248F939F93EF93FF938091DB09E82F00
:10580000F0E09091C600E65AF64F90838F5F809348
:10581000DB098091DB09803811F41092DB09FF91DC
:10582000EF919F918F910F900BBE0F900FBE0F9035
:105830001F901895CF93DF93EC0108C08A3019F4BC
:105840008DE00E94812B89910E94812B8881882381
:10585000A9F7DF91CF9108951F93CF93DF93EC01C8
:105860002196FC0114911A3019F48DE00E94812BCD
:10587000812F0E94812BFE0121961491112399F70B
:10588000DF91CF911F9108950F931F93CF93DF93D3
:10589000082FC8E0D0E010E8812F802311F081E3C9
:1058A00001C080E30E94812B16952197A9F7DF9113
:1058B000CF911F910F910895DF92EF92FF920F9376
:1058C0001F93CF93DF93CDB7DEB729970FB6F89428
:1058D000DEBF0FBECDBF8C01DE011196E8EBF3E019
:1058E00088E001900D928150E1F77E010894E11C5F
:1058F000F11C84E0D82E91E010C08F5F021B130BC7
:1059000090E002171307C8F7992329F4805D99875F
:105910000E94812B9985DA9431F0F7012191319120
:105920007F0180E0EECF802F805D0E94812B299641
:105930000FB6F894DEBF0FBECDBFDF91CF911F91A0
:105940000F91FF90EF90DF9008951F93CF93DF9317
:10595000CDB7DEB760970FB6F894DEBF0FBECDBFF0
:10596000182FDE011196E0ECF3E080E101900D923A
:105970008150E1F7812F82958F70E1E0F0E0EC0F2C
:10598000FD1FE80FF11D80810E94812B1F70E1E057
:10599000F0E0EC0FFD1FE10FF11D80810E94812BD3
:1059A00060960FB6F894DEBF0FBECDBFDF91CF91EA
:1059B0001F910895CF93DF93CDB7DEB7C354D04086
:1059C0000FB6F894DEBF0FBECDBF1092E30880E89B
:1059D00080BFA89528E288E190E00FB6F894A895DA
:1059E000809360000FBE209360001092E708109231
:1059F000E8081092E9081092EA081092ED080E9457
:105A0000702B0E9493080E945C2A0E944120909370
:105A1000F2088093F10889E0809381008FE39FE191
:105A2000909389008093880082E080936F002C9887
:105A300085B1806685B984B1806784B94098389A09
:105A4000139A149881B1886181B915980D9A469876
:105A50003E9A5A9A5B9880E060E14FE154E027E279
:105A600034E00E941E1181E060E24FE054E027E341
:105A700034E00E941E1182E060E447E154E02FE22E
:105A800034E00E941E111092EB0878948FEF9FE093
:105A90000E94F22F082F8F3F31F48FEF9FE060E0DC
:105AA0000E94043000E080EE93E00E942C2C88EFEE
:105AB00093E00E942C2C802F0E94A52C87E094E07C
:105AC0000E942C2C82B18C7F82B900FD119A01FDBD
:105AD000109A1092E6088BE193E00E941A2C0E9423
:105AE000D30E0E945C2C89E094E00E942C2C8BE069
:105AF00094E00E942C2C809160000E94A52C84E1EF
:105B000094E00E942C2C86E194E00E942C2C82E3ED
:105B100093E00E941A2C8FE194E00E942C2C85E3E4
:105B200094E00E942C2C8BE394E00E942C2C8BE4BC
:105B300094E00E942C2C81E594E00E942C2C8CE5B2
:105B400094E00E942C2C85E694E00E942C2C8AE69E
:105B500094E00E942C2C86E794E00E942C2C8AE78B
:105B600094E00E942C2C83E894E00E942C2C85E881
:105B700094E00E942C2C84B70E94A52C8DE894E020
:105B80000E942C2C14BE0E94F0138093EC080E94FB
:105B9000760F88E393E00E941A2C8091EC080E9413
:105BA000A52C89E493E00E941A2C0E943E0E80E20C
:105BB000809337091092380900E010E0FF24FA942E
:105BC000A8950E94770E0E945B098091E1088823C6
:105BD000B1F080E96EED78E00E944B1382E964EE4B
:105BE00078E00E944B130E944B2A8A30910528F0DE
:105BF00088E46FEE78E00E946F291092E1080E941D
:105C00002E268091E208882321F00E944E211092D6
:105C1000E2080E94860F882311F0A895FACF0E940F
:105C2000F60F8091F1089091F208FC01208120FF8D
:105C30002AC00E946514E091F108F091F208908169
:105C40009E7F90838823F9F4CF010E943214209123
:105C5000F1083091F208882389F4C901BE016F5F11
:105C60007F4F0E948C14882371F0CE0101960E9410
:105C70003814CE0101960E94FA1005C0C9010E9495
:105C800044200E9418118091EE08882309F498CFCF
:105C90000E943A2B882379F00E94412B882359F0E7
:105CA00081E08093EB080E94372B8FE894E00E94FC
:105CB0002C2C00E010E08091E7089091E808A0917A
:105CC000E908B091EA080196A11DB11D8093E7088B
:105CD0009093E808A093E908B093EA0880E00E9456
:105CE000D51181E00E94D51182E00E94D5118091EA
:105CF000EB08843009F460C0853040F48130E9F06D
:105D0000813070F0833009F0A2C037C0863009F4CA
:105D10008CC0863008F471C0873009F098C087C005
:105D200081B18C7F81B98AB1837F8AB90D9A389A03
:105D3000139A14981092ED088AC080E00E94070917
:105D4000F2E08C3B9F0708F482C00F5F1F4F0230C8
:105D5000110509F07CC083E08093EB081398149A36
:105D600089EA94E00E942C2C8091E7089091E80841
:105D70000E945C2C82ED94E01CC00530110519F4E2
:105D800081B1836081B90F5F1F4F0531110508F4A0
:105D90005EC0389884E08093EB0885ED94E00E9423
:105DA0002C2C8091E7089091E8080E945C2C85E0FB
:105DB00095E00E942C2C49C0319B49C081E0809322
:105DC000E3080F5F1F4F0630110508F440C00D981F
:105DD0008AB18C608AB985E08093EB0888E095E011
:105DE0000E942C2C8091E7089091E8080E945C2C7E
:105DF00086E395E00E942C2C2AC08091ED08882330
:105E000031F589E395E00E942C2C8091E708909170
:105E1000E8080E945C2C8CE495E00E942C2C0E94E7
:105E2000090F81E08093ED0812C00D9A10C0389AD6
:105E30000D9A8AB1837F8AB9139A149881E080936E
:105E4000E6081092EB081092ED0800E010E0E090F8
:105E5000EB08FE1409F441C022E0E216B9F02E1559
:105E600030F081E0EE2071F0E816B9F50AC0E5E007
:105E7000EE16E1F0F7E0EF1621F124E0E21669F505
:105E80000AC081E060E041E050E01FC081E060E0D6
:105E900042E050E01AC081E060E040E050E00E9443
:105EA000381182E060E042E050E015C081E060E03F
:105EB00040E050E00E94381182E060E041E050E0B4
:105EC0000AC081E060E040E050E00E94381182E0CA
:105ED00060E040E050E00E9438111092EE08FE2C85
:105EE0006FCE629FD001739FF001829FE00DF11D84
:105EF000649FE00DF11D929FF00D839FF00D749F44
:105F0000F00D659FF00D9927729FB00DE11DF91FEF
:105F1000639FB00DE11DF91FBD01CF01112408954C
:105F2000991B79E004C0991F961708F0961B881FEB
:105F30007A95C9F78095089597FB092E07260AD010
:105F400077FD04D00CD006D000201AF4709561952E
:105F50007F4F0895F6F7909581959F4F0895AA1B5E
:105F6000BB1B51E107C0AA1FBB1FA617B70710F044
:105F7000A61BB70B881F991F5A95A9F78095909576
:105F8000BC01CD010895FB01DC0102C005900D921A
:105F900041505040D8F70895FB01DC0104C08D91B9
:105FA0000190801921F441505040C8F7881B990B8B
:105FB0000895FB01DC0102C001900D924150504058
:105FC000D8F70895DC01CB01FC01F999FECF06C09A
:105FD000F2BDE1BDF89A319600B40D9241505040A7
:105FE000B8F70895F999FECF92BD81BDF89A992727
:105FF00080B50895DC01CB0103C02D910E940530CE
:1060000041505040D0F70895262FF999FECF1FBA7E
:1060100092BD81BD20BD0FB6F894FA9AF99A0FBED1
:0860200001960895F894FFCFEA
:106028000A0001FFFF204552524F5221003A20300A
:1060380078000A002E2E2E204552524F52210A0077
:106048002E2E2E20646F6E65210A00646F6E652106
:106058000A00205265616420556E697175652D4985
:10606800443A200020525F4552524F522100206D81
:10607800560A0020000A0A383330303E0A00756E8E
:106088006B6E6F776E20636F6D6D616E640A00389A
:106098003330303E00535441540048454C50005270
:1060A800544D310052544D320052544D3300525425
:1060B8004D340052544D350052544D360052544D13
:1060C800370052544D3800564F4C540050524F4DE3
:1060D800004944004441435700444143520000757D
:1060E80002F20D7A02060C7F02CB0D8402A40D8900
:1060F80002920D8E02890D9302800D9802770D9DF4
:1061080002000CA202380DA702E20CAC02860CB108
:1061180002A00CB402370CB9020C0CBE0200000A33
:1061280000726571206F75742064726F7070656499
:1061380020616674657220330A000A4D6F64756CBD
:10614800652053657269616C204E756D6265723A9F
:106158002000322E372E33004D6F64756C65204158
:106168006464726573733A20000A0A000A006F6655
:1061780066733A0020636E743A002000322E372E80
:10618800330044062A069B07EA055B071B07DB0664
:10619800AA056A059B065B060A0072746D20636D8A
:1061A8006E206864722063686B206661696C0A00FF
:1061B8006D756C74206865616465722063686563D9
:1061C8006B73756D206572726F72210A0020002052
:1061D800002FFC2C1C06FFFF1027E80364000A00B0
:1061E8003031323334353637383941424344454605
:00000001FF
